:10000000EBEF03F01200000004EF04F01200120006
:100018000CEF04F012000F6A1E0E716E0401400E00
:10002800096F200E0A6F040E0B6F880E086F04010B
:10003800200E0E6F040E0F6F400E0C6F1200550E3F
:10004800A76EAA0EA76EA68212000D6A040121519E
:100058000D5C1CE2156A166A22510D24F36E2351B9
:100068001520F46E24511620F86EF4CFF7FFF3CF65
:10007800F6FF0800F5500E6E0D50EA6A250FE96E7E
:10008800040EEA220EC0EFFF0D2AE0D7F86A12002C
:10009800F00E04012217840EA66E0D6A0401215188
:1000A8000D5C23E20D50EA6A250FE96E040EEA2280
:1000B800EFCF17F00D50146E156A166A22510D24F1
:1000C800F36E23511520F46E24511620F86EF4CFE8
:1000D800F7FFF3CFF6FF17C0F5FF0C000F0E0D1456
:1000E8000F0801E1ACDF0D2AD9D71200940EA66ED5
:1000F8000D6A040121510D5C1DE20D50146E156A44
:10010800060ED89014361536E804FBE1166A15BEBB
:100118001668040122511424F36E23511520F46E3D
:1001280024511620F86EF4CFF7FFF3CFF6FF87DFE0
:100138000D2ADFD7F86A1200A66A0D6A0401215158
:100148000D5C0EE222510D24A96EA6800D50EA6ABC
:10015800250FE96E040EEA22A8CFEFFF0D2AEED78D
:1001680012000D6A040121510D5C12E222510D2486
:10017800A96E0D50EA6A250FE96E040EEA22EF50C7
:10018800A86E040EA66E5BDFA6B2FED70D2AEAD7CC
:100198001200C40EA66E0D6A040121510D5C1FE207
:1001A8000D50EA6A250FE96E040EEA22EFCF17F028
:1001B8000D50146E156A166A22510D24F36E2351E0
:1001C8001520F46E24511620F86EF4CFF7FFF3CF04
:1001D800F6FF17C0F5FF0C0032DF0D2ADDD7F86AED
:1001E80012007ED8060E015C03E36D50020B01E09D
:1001F80076D00F0410E104010CBF0CD00401400EAE
:10020800096F400E040108170401087D880E0401D7
:1002180008130F6A64D0040108BF61D00D6A040195
:100228002051320A40E0CD0A32E0F80A2CE0020AF6
:1002380026E0010A20E0070A1AE0010A14E0030A8E
:100248000EE0070A0CE0060A01E03AD00401140E99
:10025800226F0401010E236F040E0D6E32D0F5DEFD
:10026800050E0D262ED014DF010E0D6E2AD03EDFAE
:10027800010E0D6E26D060DF050E0D2622D071DF2F
:10028800010E0D6E1ED085DF010E0D6E1AD06D9613
:10029800106A116A1006000E115A1050111001E070
:1002A800F9D7FF000ED0030E0401215D02E1010E13
:1002B8000D6E040E0401215D02E1010E0D6E01D0E8
:1002C80000D0010E0F6E0D500AE00DC00DF4400E67
:1002D80004010C1704010C7D880E04010C13120094
:1002E8001250131004E1200E126E4E0E136E1206F9
:1002F800000E135A6DA208D0125013102CE18B7007
:100308008B50010B24E121D00150060A17E0050AA1
:1003180013E0010A0FE0070A08E0040A04E0010AF2
:1003280018E18B9012D08B8012D01250131013E169
:100338008B700BD08B8009D08B9009D01250131082
:100348000AE18B708B50010B02E08B9212008B82BA
:1003580012008B808B8212006C5035E10401005131
:100368003C0BE842E8420D082CE10401049F180EFA
:100378000401021924E1040E031921E1100E026F91
:10038800040E036F00016A6B6A51146E156A080E39
:10039800145C000E155813E26A51EA6A180FE96EE8
:1003A800040EEA22EF50E66E6A51EA6A100FE96E0F
:1003B800040EEA22E552E750EF6E6A2BE5D7ECEF20
:1003C80001F0F4EF01F0040E6C5C01E124D8120096
:1003D800056A066A0B6A0C6A03EC03F061EF02F027
:1003E800020E055C0DE10401180E026F040E036F86
:1003F800080E016F00BD02D0C80E0BD0880E09D0C0
:100408009AD80401080E016F100E026F040E036FD4
:100418008C0E006F1200040E015C09E112C46EFF1D
:100428006E50000802E2050E01D0030E016E0504AD
:1004380009E10AD8040104BD02D0C80E01D0880E13
:10044800046F12009FEF02F0080E0B5C000E0C58B0
:1004580003E20BC06CF003D00001080E6C6F6CC097
:1004680005F400016C51146E156A14500B5E15509A
:100478000C5A180E096E040E0A6E6C511DE002A289
:1004880007D007C0F6FF08C0F7FF0800F55005D0F1
:1004980007C0E9FF08C0EAFFEF50E66E09C0E9FFB0
:1004A8000AC0EAFFE552E750EF6E072A000E08225D
:1004B800092A0A226C07E1D712006D9806500BE151
:1004C8000401080E016F100E026F040E036F840EF4
:1004D800006F04011ED0040110AF1DD00B50165D33
:1004E8000C50175904E216C40BF017C40CF0ACDF1B
:1004F800010E056E0401080E016F100E026F040E46
:10050800036F800E006F0401180E066F040E076F4C
:10051800C80E046F1200020E056E0401056BC80EAA
:10052800046F0401080E016F180E026F040E036FAA
:10053800C80E006F1200056A0401046B1200080E51
:100548006D6E6DBAFED7686A110E696E020E016E85
:1005580012006850040B09E06950040B06E06D9224
:10056800699468A402D06894FCD76850010B04E031
:100578006950010B01E024D86850100B0AE069505B
:10058800100B07E0698468986D82A19AA08A03001D
:10059800A19A6850200B06E06950200B03E070B068
:1005A8007090689A030E015C01E209D06850080B4C
:1005B80006E06950080B03E0B0EC01F06896120001
:1005C800686A7B0E696E6E6A160E706E68A605D034
:1005D800689600D000D00000F9D76D989FEC02F023
:1005E8000401080E016F0401100E026F040E036F60
:1005F80004018C0E006F036A030E016E12000401E1
:100608001051600BE842E842E842E842E84200093B
:1006180001E012001151080A2FE0010A2BE00F0A2D
:1006280008E0030A01E01200010E066E040E016ED6
:100638001200010E066E130506E14E0E076E070E38
:10064800086E120E11D0020E135D06E1600E076EE1
:10065800070E086E200E08D0030E135D08E1800E09
:10066800076E070E086E040E0B6E0C6A01D0066A40
:10067800028212004AEF03F0010E066E030E076EA7
:10068800000E086E0292010E0B6E1200010E066E2D
:1006980012C403F00401125103E1050E016E1200A9
:1006A800060E016E0FEF00F0060EF66E000EF76EE6
:1006B800000EF86E00010900F550656F0900F5504D
:1006C800666F03E1656701D03DD00900F550606FA2
:1006D8000900F550616F0900F550626F09000900C3
:1006E800F550E96E0900F550EA6E090009000900A5
:1006F800F550636F0900F550646F09000900F6CFE3
:1007080067F0F7CF68F0F8CF69F060C0F6FF61C016
:10071800F7FF62C0F8FF0001635302E1645307E08A
:100728000900F550EE6E6307F8E26407F9D767C071
:10073800F6FF68C0F7FF69C0F8FF00016507000E03
:10074800665BBFD712001201000200000008D8043F
:100758000B000100000000010902200001010080D7
:10076800320904000002FFFFFF00070501024000F4
:10077800000705810240000004030904C150006E0F
:100788000F0EC11282A404D00050C16E00EF04F015
:100798008B6AFC0E946E126A136A140E6F6EA3ECC9
:1007A80002F0ADEC02F0F5EC00F0FBD71200000E01
:1007B800F36E00EE00F0080E01D81200EA6002D0D5
:1007C800EE6AFCD7F350E9601200EE6AFCD713EE2C
:1007D80000F023EE00F0F86A199C58EC03F007ECDF
:0A07E80000F0C2EC03F0FBD7120092
:10080000D6EF2BF012001200E4EF05F01200FEFF0D
:100818001CEF04F0120002000E080000F4010000B2
:10082800020000000B580000800200004E0000008B
:10083800D8CFE4FFE0CFE4FFE46EDACFE4FFE2CF05
:10084800DAFFE9CFE4FFEACFE4FFF6CFE4FFF7CF22
:10085800E4FFF5CFE4FFF3CFE4FFF4CFE4FFFACFF2
:10086800E4FF00EE1AF0140EE80403E3EECFE4FF11
:10087800FBD700EE2EF0100EE80403E3EECFE4FF02
:10088800FBD7E6524EEC17F09EA200D19E92030EC3
:100898003E6E0E50EA6A510FE96E010EEA22EF50E1
:1008A8003E5C30E10E50E96EEA6AD890E936EA36E5
:1008B800690EE926010EEA22EECF3EF0EFCF3FF0B7
:1008C8003FC03EF03F6A3E50D76E0E50E96EEA6A6E
:1008D800D890E936EA36690EE926010EEA22EECF0B
:1008E8003EF0EFCF3FF03E50D66EF28AF294D58EAE
:1008F8000E50EA6A510FE96E010EEA22040EEF6EFD
:100908000E50106E020E3E6E0F50EA6A510FE96EDD
:10091800010EEA22EF503E5C49E10F50E96EEA6AA7
:10092800D890E936EA36690EE926010EEA22EE5039
:10093800ED1009E10F50EA6A510FE96E010EEA2243
:10094800010EEF6E33D0080E0F5C0CE2070E0F1489
:100958003E6E010E3E5204E0E846FE0B3E06FCE108
:1009680089121AD0100E0F5C0CE2070E0F143E6E9F
:10097800010E3E5204E0E846FE0B3E06FCE18A12F8
:100988000BD0070E0F143E6E010E3E5204E0E846EF
:10099800FE0B3E06FCE18B120F50EA6A510FE96E1E
:1009A800010EEA22030EEF6E0F500E6E0F2A060E8E
:1009B8000F5C02E1080E04D0130E0F5C03E1160E63
:1009C8000F6E04D0180E0F5C01E10F6A000ED8807C
:1009D8000254000E03542EE2112A000E1222025075
:1009E800115C0350125826E3116A126A030E065C62
:1009F8001FE20450EA6A480FE96E010EEA2280CF2E
:100A0800EFFF0450EA6A4B0FE96E010EEA2281CF2C
:100A1800EFFF0450EA6A4E0FE96E010EEA2282CF18
:100A2800EFFF042A030E045C01E3046A062A02D0DD
:100A3800026A036A000ED8800754000E085419E2AF
:100A48000C50000816E2132A000E14220750135CFB
:100A5800085014580EE3136A146A030E0B5C07E27D
:100A6800092A030E095C01E3096A0B2A02D0076A06
:100A7800086A0C5000080AE2156A1550040DF3289C
:100A8800C26E9E9C9F9C9D8CC280C2829EAC2BD0C5
:100A98009E9CC450436E426AC35000014210406E8F
:100AA80043C041F01550060DF3CF3EF0F4CF3FF0B0
:100AB800000E3E26010E3F220950020D3E50F3243F
:100AC800E96E3F50F420EA6E40C0EEFF41C0EDFFF2
:100AD800152A0C50155C02E39D9C05D01550040D99
:100AE800F328C26EC282F2A442D0D59EF294F29A42
:100AF800040E3E6E1050EA6A510FE96E010EEA22AA
:100B0800EF503E5C34E1080E105C0DE2070E101445
:100B18003E6E010E3E5204E0E846FE0B3E06FCE146
:100B2800E81C89161CD0100E105C0DE2070E10147C
:100B38003E6E010E3E5204E0E846FE0B3E06FCE126
:100B4800E81C8A160CD0070E10143E6E010E3E5299
:100B580004E0E846FE0B3E06FCE1E81C8B1610504C
:100B6800EA6A510FE96E010EEA22020EEF6EE552B3
:100B780000EE3DF0100EE80403E3E5CFEDFFFBD7F0
:100B880000EE2DF0140EE80403E3E5CFEDFFFBD7EC
:100B9800E5CFFAFFE5CFF4FFE5CFF3FFE5CFF5FFAB
:100BA800E5CFF7FFE5CFF6FFE5CFEAFFE5CFE9FFB1
:100BB800E5CFDAFFE550E5CFE0FFE5CFD8FF10003D
:100BC800DACFE4FFE652A1A211D01650B36E175047
:100BD800B26E192A1850195C08E302018051891A6B
:100BE80081518A1A82518B1A196AA192E552E5CF6E
:100BF800DAFF1100D9CFE6FFE1CFD9FF020EE126D7
:100C0800896A92680F0EC16EC2900C6A070EB46EA4
:100C18008A6A93688B6A94688B908B92949094926A
:100C280094840101010EE66F0101F469F5690A6A0D
:100C3800096A0B6A056A046A066A026A036A076A2D
:100C4800086A116A126A136A146A156ACA82CA8023
:100C5800CA9CCA9ACA88CA96FA0ECB6EDF6ADFCFD8
:100C68002EF00C0EE76E2E18E8AE02D0E73402D054
:100C7800E7502E5C36E2010EDB6ADBCF2EF0030E66
:100C8800E76E2E18E8AE02D0E73402D0E7502E5CAB
:100C980026E2DFCF2EF02F6A2EBE2F68060E2F0217
:100CA800F3CF2FF02E02F3CF2EF0F4502F26000EA4
:100CB8002E26010E2F22010EDBCF30F0316A30BE16
:100CC8003168D890303631362E503024E96E2F50A6
:100CD8003120EA6EEE6AED6A010EDB2ACED7DF2AF2
:100CE800BED70101E06BE16BDE6BDF6BE26BE36BA0
:100CF800E46BE56B0E6A0F6A106ADF6ADFCF2EF0CD
:100D0800180EE76E2E18E8AE02D0E73402D0E7508E
:100D18002E5C1BE2DFCFE9FFEA6AE9BEEA68D890F9
:100D2800E936EA36690EE926010EEA22EE6AED6A2C
:100D3800DFCFE9FFEA6AE9BEEA68510EE926010E4B
:100D4800EA22010EEF6EDF2AD9D7D586D59AD59C2F
:100D5800F294F29AF194D08ECA949D829F92F28E68
:100D6800F28CCA84020EE15C02E2E16AE552E16EAD
:100D7800E552E7CFD9FF1200D9CFE6FFE1CFD9FF7F
:100D8800050EE126020EDB6A030EDB6A040EDB6A3F
:100D980052EC16F00650000809E254EC0CF0052A53
:100DA800030E055C01E1056A0606F4D70B5000083E
:100DB80009E27EEC0CF00A2A030E0A5C01E10A6AD9
:100DC8000B06F4D7200E0001E76E6019E8AE02D0DA
:100DD800E73402D0E750605D01E2A5D16D50020B07
:100DE80001E0A1D1400EE66E400EE66E020EE66E00
:100DF8005DEC26F0E552E552E552E76E030EE7CFCB
:100E0800DBFFDB50000801E324D1040EDB6A030E8C
:100E1800DB50F36E040EDBCFF4FFF350F45C01E318
:100E280018D1040EDB50EA6A400FE96E020EEA227E
:100E3800EFCFDFFF0201C75141E10D0E2E6EDF50EB
:100E48002E5C05E00A0E2F6EDF502F5C37E1010E95
:100E5800C76F0101E051EA6A000FE96E030EEA224A
:100E68000D0EEF6EE02B010EDB6AE051F36E010E02
:100E7800DBCFF4FFF350F45C1CE2010EDBCFE9FF9B
:100E8800EA6AE9BEEA68000EE926030EEA22EF5094
:100E9800E66E010EDBCFE9FFEA6AE9BEEA68830E77
:100EA800E926020EEA22E552E750EF6E010EDB2A30
:100EB800DCD7C1D90101E06BE16BBBD01B0EDF5C55
:100EC80009E1C35107E1010EC36F1B0EC46FC56B67
:100ED800C66BAFD0C3050BE15B0EDF5C08E11B0EF0
:100EE800C45D05E1C55103E15B0EC56FA2D0C30522
:100EF80066E1410EDF5C63E11B0EC45D60E15B0EE1
:100F0800C55D5DE1C46BC56BC66BC36B010EDB6A67
:100F1800DBCFE9FFEA6AE9BEEA68000EE926030EBC
:100F2800EA22EF500D081CE0010EDBCFE9FFEA6A68
:100F3800E9BEEA68830EE926020EEA22EF50E66E61
:100F4800010EDBCFE9FFEA6AE9BEEA68000EE9268E
:100F5800030EEA22E552E750EF6E010EDB2AD8D7DE
:100F6800010EDBCFE0F10101E051EA6A000FE96E02
:100F7800030EEA22EF6A4D0E2E6E510E2F6E306A66
:100F88002EC0E6FFE66E30C0E6FF64EC2AF0E552BC
:100F9800E552E552000EE66E030EE66E4A0E2E6E20
:100FA800510E2F6E306A2EC0E6FFE66E30C0E6FFA7
:100FB80064EC2AF0316E050EE15E31503AD0080E2D
:100FC800DF5C1CE10101E051000818E2E007E05194
:100FD800EA6A000FE96E030EEA22EF6A470E2E6EE8
:100FE800510E2F6E306A2EC0E6FFE66E30C0E6FF67
:100FF80064EC2AF0E552E552E5521BD00D0EDF5C99
:1010080018E00A0EDF5C15E0200EDF5C12E3020137
:10101800C46BC56BC66BC36B0101E051EA6A000F74
:10102800E96E030EEA22DFCFEFFF0201C76B010171
:10103800E02B0101E0512E6E2F6A000E2E1806E1FA
:10104800010E2F1803E10D86E06BE16B040EDB2A1D
:10105800DED60D5067E00DA00FD0410E2E6E510E5A
:101068002F6E306A2EC0E6FFE66E30C0E6FF64ECF5
:101078002AF0E552E552E5520DA40FD0250E2E6E4A
:10108800510E2F6E306A2EC0E6FFE66E30C0E6FFC6
:1010980064EC2AF0E552E552E5520DA60FD0090E90
:1010A8002E6E510E2F6E306A2EC0E6FFE66E30C0EF
:1010B800E6FF64EC2AF0E552E552E5520DA80FD0A0
:1010C800EA0E2E6E500E2F6E306A2EC0E6FFE66EC8
:1010D80030C0E6FF64EC2AF0E552E552E5520DAC6B
:1010E8000FD0C90E2E6E500E2F6E306A2EC0E6FF3E
:1010F800E66E30C0E6FF64EC2AF0E552E552E552B0
:101108000DAE0FD0B00E2E6E500E2F6E306A2EC060
:10111800E6FFE66E30C0E6FF64EC2AF0E552E552E1
:10112800E5520D6A3FD8050EE15C02E2E16AE5523C
:10113800E16EE552E7CFD9FF1200D9CFE6FFE1CF44
:10114800D9FFE652DEC1DFFFDF2A400E2E6EDF50E8
:101158002E5C01E1DF6A0101DF51DF5C01E122D889
:101168000101DE51EA6A000FE96E020EEA22FE0E64
:10117800DBCFEFFFDE2B400EDE5D01E1DE6BDF51E2
:10118800DE5D01E10D84FE0EDBCF2EF02F6A2EBE50
:101198002F682EC0F3FF2FC0F4FFE552E552E7CFCA
:1011A800D9FF1200D9CFE6FFE1CFD9FFE6520101FE
:1011B800DE51DF5D3BE00201CF5103E05BEC27F03D
:1011C800FAD70101DF51D880DE5517E2DF51DE5D25
:1011D800DF6EDFCFE6FFDF512F6A000F2E6E020EA3
:1011E8002F222EC0E6FF2FC0E6FFBDEC26F0E55209
:1011F800E552E552DEC1DFF117D0400ED880DF5549
:10120800DF6EDFCFE6FFDF512F6A000F2E6E020E72
:101218002F222EC0E6FF2FC0E6FFBDEC26F0E552D8
:10122800E552E5520101DF6B5BEC27F0E552E55230
:10123800E7CFD9FF1200D9CFE6FFE1CFD9FF040EDF
:10124800E126DE6ADD6A020EDB6A030EDB6A010153
:10125800E151EA6A000FE96E030EEA22EF50E66EEA
:10126800E66A6BEC2BF0E552E552020EF3CFDBFF9A
:101278000101E12BE1512E6E2F6A000E2E1804E1B8
:10128800010E2F1801E1E16B020EDB50DE6EDD6A04
:10129800E151EA6A000FE96E030EEA22EF502C08CA
:1012A80036E0E151EA6A000FE96E030EEA22EF50D8
:1012B8000D082DE0E151EA6A000FE96E030EEA22FB
:1012C800EF50E66EE66A6BEC2BF0E552E552030E42
:1012D800F3CFDBFF0101E12BE1512E6E2F6A000EE7
:1012E8002E1804E1010E2F1801E1E16B020EDBCF8D
:1012F80030F030C031F0306A030EDB50000130248A
:101308002E6E000E31202F6E2EC0DEFFDD6E000E19
:10131800DFCF22F0010EDBCF23F0460E221801E1C9
:10132800235001E1FDD0490E221802E1430E231893
:1013380001E1F3D0490E221802E1520E231801E10F
:10134800E9D0490E221802E1530E231801E1DFD03B
:10135800530E221802E1430E231801E1D5D0530E93
:10136800221802E1520E231801E1CBD0530E2218A5
:1013780002E1530E231801E1C1D0530E221802E1F5
:10138800420E231801E1B7D0430E221802E1420EA3
:10139800231801E1ADD0430E221802E1520E2318A2
:1013A80001E1A3D04F0E221802E1420E231801E1F9
:1013B80099D0570E221802E14D0E231801E190D062
:1013C800520E221802E14D0E231801E187D0440E77
:1013D800221802E1500E231801E17ED04F0E221888
:1013E80002E1500E231875E0490E221802E1500E52
:1013F80023186DE0580E221802E1540E231864E0F9
:10140800540E221801E123505DE0410E221801E13B
:10141800235056E0560E221801E123504FE0490EA2
:10142800221801E1235048E04F0E221801E1235011
:1014380041E0550E221802E1430E231839E0580EF8
:10144800221802E1430E231830E0430E221801E16E
:10145800235029E0520E221801E1235022E0580EB1
:10146800221802E1520E231819E0030EDB505BE14B
:10147800020EDBCFE6FFE66ADBCFE6FFE66A8D0EFB
:101488002E6E500E2F6E306A2EC0E6FFE66E30C00C
:10149800E6FF64EC2AF0316E070E63D02DEC0FF0F6
:1014A80062D097D860D02CD95ED02FEC0FF05BD0EB
:1014B80094D859D09CD957D0F3D955D00BDA53D0FA
:1014C80019DA51D0D2D84FD02BEC0FF04CD094DB96
:1014D8004AD085EC0EF047D0EADA45D0A6DA43D0F8
:1014E80066DA41D04CEC10F03ED031EC0FF03BD036
:1014F800E4EC0FF038D0A5EC11F035D074EC12F014
:1015080032D076EC12F02FD078EC12F02CD07AECA6
:1015180012F029D07CEC12F026D07EEC12F023D009
:1015280080EC12F020D0030EDBCFE6FFE66A020E55
:10153800DBCFE6FFE66A030EDBCFE6FFE66A020EC4
:10154800DBCFE6FFE66A650E2E6E500E2F6E306A10
:101558002EC0E6FFE66E30C0E6FF64EC2AF0316E7E
:101568000B0EE15E31500101E151EA6A000FE96EAC
:10157800030EEA22EF500D080DE00D500BE1520E5C
:101588002E6E2F6ADF502E1803E1DE52DD502F1821
:1015980001E00D8EE0C1E1F1040EE15C02E2E16AD6
:1015A800E552E16EE552E7CFD9FF12000101E6519D
:1015B8000FE06A0E2E6E570E2F6E306A2EC0E6FFB1
:1015C800E66E30C0E6FF64EC2AF0E552E552E552DB
:1015D8001200FEEC05F0DAEF0AF0D9CFE6FFE1CF12
:1015E800D9FF030EE126E66AD9CFE6FFDACFE6FF98
:1015F800010EE66EE7EC13F0E552E552E552E552CE
:10160800E66AD950010FE66E000EDA20E66E020E89
:10161800E66EE7EC13F0E552E552E552E5520D505F
:101628001AE1DF0417E1D950010FE96EDACFEAFFBA
:10163800EE50ED100AE0010E2E6E2F6ADB502E18C8
:1016480008E1020EDB502F1804E1010EDBCFE6F1B2
:1016580001D00D8CABDF030EE15C02E2E16AE552DA
:10166800E16EE552E7CFD9FF1200D9CFE6FFE1CF0F
:10167800D9FF030EE126020EDB6AE66A000EE66E6B
:10168800000EE66E030EE66EE7EC13F0E552E55247
:10169800E552E552E66AD950020FE66E000EDA20EE
:1016A800E66E010EE66EE7EC13F0E552E552E55200
:1016B800E5520D501BE1020EDB500CE10050011009
:1016C80003E1026A036A11D0CA8400C002F001C0B3
:1016D80003F00BD00050011003E1076A086A05D037
:1016E800CA8400C007F001C008F060DF030EE15CA7
:1016F80002E2E16AE552E16EE552E7CFD9FF120056
:10170800D9CFE6FFE1CFD9FF040EE126E66AD9CFAB
:10171800E6FFDACFE6FF010EE66EE7EC13F0E552DE
:10172800E552E552E552E66AD950010FE66E000E21
:10173800DA20E66E010EE66EE7EC13F0E552E552AC
:10174800E552E552E66AD950020FE66E000EDA203D
:10175800E66E010EE66EE7EC13F0E552E552E5524F
:10176800E552E66AD950030FE66E000EDA20E66EFF
:10177800010EE66EE7EC13F0E552E552E552E5524C
:101788000D502BE1DF50926E010EDB50936E020E6E
:10179800DB50946E030EDB500D0805E20D0EF36E60
:1017A800030EF3CFDBFF030EDB5005E10F0EC16E16
:1017B800C2900C6A11D00C6AC26A030EDBCFE6FF36
:1017C8000F0EE552D880E754C16EBE0EC06EC280BF
:1017D800030EDB500C6ECA84E9DE040EE15C02E203
:1017E800E16AE552E16EE552E7CFD9FF1200D9CFA1
:1017F800E6FFE1CFD9FF020EE126E66AD9CFE6FF80
:10180800DACFE6FF010EE66EE7EC13F0E552E5529B
:10181800E552E552E76E010EE7CFDBFF0D5036E1EA
:10182800010EDB5002E1DF50896E010EE66ED9CF62
:10183800E6FFDACFE6FFE66EE7EC13F0E552E55295
:10184800E552E552E76E010EE7CFDBFF0D501EE1D2
:10185800010EDB5002E1DF508A6E010EE66ED9CF31
:10186800E6FFDACFE6FFE66EE7EC13F0E552E55265
:10187800E552E552E76E010EE7CFDBFF0D5006E1BA
:10188800010EDB5002E1DF508B6E90DE020EE15C50
:1018980002E2E16AE552E16EE552E7CFD9FF1200B4
:1018A8008250E66EE66A8150E66EE66A8050E66E21
:1018B800E66A520E2E6E500E2F6E306A2EC0E6FF6C
:1018C800E66E30C0E6FF64EC2AF0316E090EE15E88
:1018D80031501200720E2E6E570E2F6E306A2EC0C7
:1018E800E6FFE66E30C0E6FF64EC2AF0E552E5520A
:1018F800E5521200D9CFE6FFE1CFD9FFE652DF6A01
:10190800500E2E6E500E2F6E306A2EC0E6FFE66E19
:1019180030C0E6FF64EC2AF0E552E552E552DF6A92
:101928000C50DF5C30E2DFCF2EF02F6A2EBE2F681E
:10193800060E2F02F3CF2FF02E02F3CF2EF0F45025
:101948002F26000E2E26010E2F220A50020D2E5091
:10195800F324E96E2F50F420EA6EEECFE6FFEFCFC6
:10196800E6FF4A0E306E500E316E326A30C0E6FF26
:10197800E66E32C0E6FF64EC2AF0336E050EE15ED7
:101988003350DF2ACDD76F0E2E6E570E2F6E306A6A
:101998002EC0E6FFE66E30C0E6FF64EC2AF0E552A2
:1019A800E552E552E552E552E7CFD9FF1200D9CF0B
:1019B800E6FFE1CFD9FF030EE126E66AD9CFE6FFBD
:1019C800DACFE6FFE66EE7EC13F0E552E552E552B2
:1019D800E552E66AD950020FE66E000EDA20E66E8E
:1019E800010EE66EE7EC13F0E552E552E552E552DA
:1019F8000D5011E1DECF2EF0DDCF2FF0000E2E5C62
:101A0800100E2F5807E2DECFE9FFDDCFEAFF020E06
:101A1800DBCFEFFFCBDD030EE15C02E2E16AE552CA
:101A2800E16EE552E7CFD9FF1200D9CFE6FFE1CF4B
:101A3800D9FF030EE126E66AD9CFE6FFDACFE6FF43
:101A4800E66EE7EC13F0E552E552E552E5520D502B
:101A580024E1DECF2EF0DDCF2FF0000E2E5C100E2D
:101A68002F5807E2DECFE9FFDDCFEAFF020EEFCF06
:101A7800DBFF020EDBCFE6FFE66A400E2E6E500E4D
:101A88002F6E306A2EC0E6FFE66E30C0E6FF64ECCB
:101A98002AF0316E050EE15E3150030EE15C02E280
:101AA800E16AE552E16EE552E7CFD9FF1200D9CFDE
:101AB800E6FFE1CFD9FF030EE126E66AD9CFE6FFBC
:101AC800DACFE6FF050EE66EE7EC13F0E552E552D5
:101AD800E552E552E66AD950010FE66E000EDA20AB
:101AE800E66E010EE66EE7EC13F0E552E552E552BC
:101AF800E552E66AD950020FE66E000EDA20E66E6D
:101B0800010EE66EE7EC13F0E552E552E552E552B8
:101B18000D5068E1020EDB50010861E3010EDB5055
:101B280007085DE3410E2E6EDF502E5C1AE1020EAF
:101B3800DB500CE1010EF36EDB5004E0D890F33675
:101B4800E806FCE1F350F31C92164BD0010EF36E3D
:101B5800DB5004E0D890F336E806FCE1F35092122B
:101B680040D0420E2E6EDF502E5C1AE1020EDB5082
:101B78000CE1010EF36EDB5004E0D890F336E80672
:101B8800FCE1F350F31C93162CD0010EF36EDB50DE
:101B980004E0D890F336E806FCE1F350931221D024
:101BA800430E2E6EDF502E5C1AE1020EDB500CE164
:101BB800010EF36EDB5004E0D890F336E806FCE142
:101BC800F350F31C94160DD0010EF36EDB5004E0B5
:101BD800D890F336E806FCE1F350941202D00D8C4D
:101BE80001D0E4DC030EE15C02E2E16AE552E16E59
:101BF800E552E7CFD9FF1200D9CFE6FFE1CFD9FFF1
:101C0800030EE126020EDB6AE66AD9CFE6FFDACFD9
:101C1800E6FF050EE66EE7EC13F0E552E552E552F5
:101C2800E552E66AD950010FE66E000EDA20E66E3C
:101C3800010EE66EE7EC13F0E552E552E552E55287
:101C48000D5055E1010EDB50070836E3410E2E6EAC
:101C5800DF502E5C0BE1010EF36EDB5004E0D890F0
:101C6800F336E806FCE1F35080141FD0420E2E6EC6
:101C7800DF502E5C0BE1010EF36EDB5004E0D890D0
:101C8800F336E806FCE1F35081140FD0430E2E6EB4
:101C9800DF502E5C11E1010EF36EDB5004E0D890AA
:101CA800F336E806FCE1F3508214E76E020EE7CF44
:101CB800DBFFDB5008E002D00D8C19D0010EF36E6B
:101CC800020EF3CFDBFF020EDBCFE6FFE66A370E2C
:101CD8002E6E500E2F6E306A2EC0E6FFE66E30C0B4
:101CE800E6FF64EC2AF0316E050EE15E3150030E1A
:101CF800E15C02E2E16AE552E16EE552E7CFD9FF25
:101D08001200D9CFE6FFE1CFD9FF030EE126E66A3C
:101D1800D9CFE6FFDACFE6FF050EE66EE7EC13F063
:101D2800E552E552E552E552E66AD950010FE66EF2
:101D3800000EDA20E66E010EE66EE7EC13F0E552CF
:101D4800E552E552E552E66AD950020FE66E000EFA
:101D5800DA20E66E010EE66EE7EC13F0E552E55286
:101D6800E552E5520D5069E1020EDB50010861E3CE
:101D7800010EDB5007085DE3410E2E6EDF502E5C2E
:101D88001AE1020EDB500CE1010EF36EDB5004E0A9
:101D9800D890F336E806FCE1F350F31C89164BD0D3
:101DA800010EF36EDB5004E0D890F336E806FCE150
:101DB800F350891240D0420E2E6EDF502E5C1AE18D
:101DC800020EDB500CE1010EF36EDB5004E0D890FC
:101DD800F336E806FCE1F350F31C8A162CD0010E0A
:101DE800F36EDB5004E0D890F336E806FCE1F350DC
:101DF8008A1221D0430E2E6EDF502E5C1AE1020E9D
:101E0800DB500CE1010EF36EDB5004E0D890F336A2
:101E1800E806FCE1F350F31C8B160DD0010EF36EAF
:101E2800DB5004E0D890F336E806FCE1F3508B125F
:101E380002D00D8C02D0DAEC0AF0030EE15C02E26B
:101E4800E16AE552E16EE552E7CFD9FF1200DAEF19
:101E58000AF0DAEF0AF0DAEF0AF0D9CFE6FFE1CFBD
:101E6800D9FF040EE126E66AD9CFE6FFDACFE6FF0E
:101E7800050EE66EE7EC13F0E552E552E552E55241
:101E8800E66AD950010FE66E000EDA20E66E010E02
:101E9800E66EE7EC13F0E552E552E552E552E66AE4
:101EA800D950020FE66E000EDA20E66E030EE66EDB
:101EB800E7EC13F0E552E552E552E5520D5076E1B4
:101EC800D950020FE96EDACFEAFF720ED880EE54CD
:101ED8002E0EED5441E3D950020FE96EDACFEAFF36
:101EE800EE50ED101FE031683268336A2D0EE76E50
:101EF800020EDBCF34F0030EDBCF35F0E75034268B
:101F0800000E3522366A3450315C2E6E3550325808
:101F18002F6E36503358306E020E2EC0DBFF030E84
:101F28002FC0DBFF010EDB50070816E3410E2E6EB3
:101F3800DF502E5C02E1DF6A11D0420E2E6EDF50B8
:101F48002E5C02E1080E06D0430E2E6EDF502E5C8A
:101F580003E1100EDF6E02D00D8C28D0010EDB508D
:101F6800DF24E96EEA6AD890E936EA36690EE9268E
:101F7800010EEA22020EDBCFEEFF030EDBCFEDFFF0
:101F8800010EDB50DF24EA6A510FE96E010EEA22E6
:101F9800EF040AE1010EDB50DF24EA6A510FE96E13
:101FA800010EEA22020EEF6EDAEC0AF0040EE15C92
:101FB80002E2E16AE552E16EE552E7CFD9FF12008D
:101FC800D9CFE6FFE1CFD9FF050EE126E66AD9CFE2
:101FD800E6FFDACFE6FF010EE66EF5DBE552E552E5
:101FE800E552E552E66AD950020FE66E000EDA2095
:101FF800E66E010EE66EE7DBE552E552E552E55284
:10200800E66AD950030FE66E000EDA20E66E010E7E
:10201800E66ED9DBE552E552E552E552E66AD9505B
:10202800010FE66E000EDA20E66E010EE66ECBDBDF
:10203800E552E552E552E552E66AD950040FE66EDC
:10204800000EDA20E66E010EE66EBDDBE552E552C3
:10205800E552E5520D5012E1DFCFD9F1020EDBCF88
:10206800DBF1010EDBCFDAF1030EDBCFDCF1040E7E
:10207800DBCFDDF1D9C189FFDAEC0AF0050EE15CAE
:1020880002E2E16AE552E16EE552E7CFD9FF1200BC
:10209800D9CFE6FFE1CFD9FF040EE126030EDB6AB4
:1020A8000101E151EA6A000FE96E030EEA22EF50DE
:1020B8002C081DE00101E151EA6A000FE96E030EE8
:1020C800EA22EF50E66EE66A100E2E6E500E2F6E64
:1020D800306A2EC0E6FF2FC0E6FF30C0E6FF64EC92
:1020E8002AF0316E050EE15E31500D8A20D10101D2
:1020F800E12B0101E1512E6E2F6A000E2E1802E12C
:10210800010E2F1802E10101E16BD9C189FF01011C
:10211800DA1D89142E6E891C0101DA152E10E76E5E
:10212800010EE7CFDBFF0101E151EA6A000FE96E1A
:10213800030EEA22EF500D0801E1F7D00101E15149
:10214800EA6A000FE96E030EEA22EF50E66EE66ACD
:102158006BEC2BF0E552E552020EF3CFDBFF300EAD
:10216800F36E020EDBCFF4FFF350F45C0FE3020EC4
:10217800DB5039080BE3300E2E6E020EDBCFE7FF83
:102188002E50E75E020EE7CFDBFF19D0410EF36E4B
:10219800020EDBCFF4FFF350F45C0FE3020EDB50CA
:1021A80046080BE3370E2E6E020EDBCFE7FF2E50EC
:1021B800E75E020EE7CFDBFF02D00D8CB8D0020E2F
:1021C800DB38F00BDF6E0101E12B0101E1512E6ECE
:1021D8002F6A000E2E1802E1010E2F1802E10101EC
:1021E800E16B0D0E2E6E0101E151EA6A000FE96EF6
:1021F800030EEA22EF502E5C02E10D8898D001010F
:10220800E151EA6A000FE96E030EEA22EF50E66E2A
:10221800E66A6BEC2BF0E552E552020EF3CFDBFFDA
:10222800300EF36E020EDBCFF4FFF350F45C0FE3D5
:10223800020EDB5039080BE3300E2E6E020EDBCF98
:10224800E7FF2E50E75E020EE7CFDBFF19D0410E05
:10225800F36E020EDBCFF4FFF350F45C0FE3020ED3
:10226800DB5046080BE3370E2E6E020EDBCFE7FF7E
:102278002E50E75E020EE7CFDBFF02D00D8C57D061
:10228800020EDB50DF24DF6E0101E12B0101E15179
:102298002E6E2F6A000E2E1802E1010E2F1802E191
:1022A8000101E16BDF508A6E010EDB50896E01017E
:1022B800DD5105E0DDC1E6FFF2EC2BF0E552D9C1B6
:1022C80089FF0101DC5130E0030EDCC1DBFF0101B5
:1022D800D9510101DB152E6E0101DB5180142E5CF2
:1022E8000BE1030EDB5008E00000000000000000D6
:1022F8000000030EDB06EBD7030EDCC1DBFF010198
:10230800D9510101DB152E6E0101DB5180142E5CC1
:102318000BE0030EDB5008E00000000000000000A6
:102328000000030EDB06EBD7FED6DAEC0AF0040E4B
:10233800E15C02E2E16AE552E16EE552E7CFD9FFDE
:102348001200D9CFE6FFE1CFD9FF050EE126030E33
:10235800DB6A040EDB6AE66AD950040FE66E000EEB
:10236800DA20E66E010EE66E2EDAE552E552E55207
:10237800E552040EDB5004E0040EDB50380802E29C
:102388000D8CA4D00101E151EA6A000FE96E030E39
:10239800EA22EF502C081DE00101E151EA6A000F22
:1023A800E96E030EEA22EF50E66EE66A100E2E6E14
:1023B800500E2F6E306A2EC0E6FF2FC0E6FF30C0E9
:1023C800E6FF64EC2AF0316E050EE15E31500D8AAD
:1023D8007DD00101E12B0101E1512E6E2F6A000E23
:1023E8002E1802E1010E2F1802E10101E16BD9C19B
:1023F80089FF0101DA1D89142E6E891C0101DA1585
:102408002E10E76E010EE7CFDBFF040EDB505CE019
:102418000101E151EA6A000FE96E030EEA22EFCFEB
:10242800DFFF0101E12B0101E1512E6E2F6A000E41
:102438002E1802E1010E2F1802E10101E16B040ED2
:10244800DB06DF508A6E010EDB50896E0101DD511B
:1024580005E0DDC1E6FFF2EC2BF0E552D9C189FFBA
:102468000101DC5130E0030EDCC1DBFF0101D95171
:102478000101DB152E6E0101DB5180142E5C0BE18E
:10248800030EDB5008E00000000000000000000020
:10249800030EDB06EBD7030EDCC1DBFF0101D951CC
:1024A8000101DB152E6E0101DB5180142E5C0BE05F
:1024B800030EDB5008E000000000000000000000F0
:1024C800030EDB06EBD7A1D7DAEC0AF0050EE15CC8
:1024D80002E2E16AE552E16EE552E7CFD9FF120068
:1024E800DAEF0AF0DAEF0AF0DAEF0AF0DAEF0AF0D8
:1024F800DAEF0AF0DAEF0AF0D9CFE6FFE1CFD9FF39
:10250800060EE126E66AD950020FE66E000EDA20C2
:10251800E66E030EE66E57D9E552E552E552E552EE
:10252800D950020FE96EDACFEAFFEE50ED1012E152
:10253800010EE66ED950040FE66E000EDA20E66E44
:10254800050EE66E40D9E552E552E552E552010E18
:10255800E66E0FD0E66AD950040FE66E000EDA2058
:10256800E66E050EE66E2FD9E552E552E552E552C4
:10257800E66AD950050FE66E000EDA20E66E010E07
:10258800E66E21D9E552E552E552E5520D5001E0DB
:1025980010D1D950020FE96EDACFEAFFEE50ED10F4
:1025A80003E1B190A09203D1020EDBCF2EF0030E0F
:1025B800DBCF2FF0640E2E5C000E2F5802E2800E47
:1025C80001D0010E186E050EDB50070801E2C1D0DC
:1025D80018503A6E3B6A3C6A3D6A020EDBCF36F011
:1025E800030EDBCF37F0386A396AD890363637367B
:1025F8003836393636C020F037C021F038C022F0DE
:1026080039C023F018C025F03BC026F03CC027F0A5
:102618003DC028F033EC2BF01CC032F01DC033F065
:102628001EC034F01FC035F02E6A1B0E2F6EB70E79
:10263800306E316A2EC020F02FC021F0226E31C0DA
:1026480023F01CC025F01DC026F01EC027F01FC0B7
:1026580028F0ADEC28F020C0DEFF21C0DDFFDECF82
:102668002EF0DDCF2FF0120E2E5C000E2F5804E254
:10267800120EDE6EDD6A0CD0DECF2EF0DDCF2FF02D
:10268800120E2E5E000E2F5A2EC0DEFF2FC0DDFF69
:102698000201806B816B826B410E2E6E040EDB5043
:1026A8002E5C19E1010EF36E050EDB5004E0D890A4
:1026B800F336E806FCE1F350F31C9216010EF36EB4
:1026C800050EDB5004E0D890F336E806FCE1F35041
:1026D8000201801340D0420E2E6E040EDB502E5C99
:1026E80019E1010EF36E050EDB5004E0D890F336C5
:1026F800E806FCE1F350F31C9316010EF36E050E89
:10270800DB5004E0D890F336E806FCE1F350020110
:10271800811321D0430E2E6E040EDB502E5C19E17E
:10272800010EF36E050EDB5004E0D890F336E80690
:10273800FCE1F350F31C9416010EF36E050EDB500A
:1027480004E0D890F336E806FCE1F3500201821366
:1027580002D00D8C2ED031683268336ADECF34F067
:10276800DDCF35F0366A3450315C2E6E3550325834
:102778002F6E36503358306E2EC0DEFF2FC0DDFF6F
:10278800DECF2EF0DDCF2FF02FC02EF02F6A2E5087
:10279800166EDECF2EF0DDCF2FF02E50176E196A91
:1027A800B192B198B19AA282A192A082B180DAECDA
:1027B8000AF0060EE15C02E2E16AE552E16EE552DA
:1027C800E7CFD9FF1200D9CFE6FFE1CFD9FF040E3A
:1027D800E126030EDB6A0D0E2E6E0101E151EA6A55
:1027E800000FE96E030EEA22EF502E5C05E1FB0EA6
:1027F800DB5044E10D8842D0E151EA6A000FE96EEE
:10280800030EEA22EF502C081FE0FB0EDB501AE102
:10281800E151EA6A000FE96E030EEA22EF50E66E14
:10282800E66A100E2E6E500E2F6E306A2EC0E6FF2E
:10283800E66E30C0E6FF64EC2AF0316E050EE15E0C
:1028480031500D8A020E90D1E12BE1512E6E2F6A84
:10285800000E2E1804E1010E2F1801E1E16B0D0E98
:102868002E6EE151EA6A000FE96E030EEA22EF507C
:102878002E5C06E1FB0EDB5001E10D88030E74D1DE
:102888002D0E2E6EE151EA6A000FE96E030EEA2260
:10289800EF502E5C27E1040E2F6EFE0EDB502F5CEE
:1028A80021E0050E306EFE0EDB50305C1BE0FE0EA4
:1028B800DB0401E12FD1030E2E6EFE0EDB502E5CE1
:1028C80001E128D1010EF36E030EF3CFDBFFE12BFC
:1028D800E1512E6E2F6A000E2E1804E1010E2F18FA
:1028E80001E1E16B040E2E6EFE0EDB502E5C11E052
:1028F800050E2F6EFE0EDB502F5C0BE0050EE66E0C
:10290800D9CFE6FFDACFE6FF3BD9E552E552E552EB
:102918003DD0E151EA6A000FE96E030EEA22EFCFDB
:102928002EF02F6A306A2EC0DFFF010E2FC0DBFFAA
:10293800020E30C0DBFF050E2E6EFE0EDB502E5C45
:1029480019E1000EDFCFE6FF010EDBCFE6FF6BECEF
:102958002BF0E552E552F3CF2EF0F4CF2FF0306A8A
:102968002FBE30682EC0DFFF010E2FC0DBFF020E26
:1029780030C0DBFF0101E12BE1512E6E2F6A000E02
:102988002E1804E1010E2F1801E1E16B030EDB5054
:102998001DE0DFCF2EF0010EDBCF2FF0020EDBCFD4
:1029A80030F02668276828682EC021F02FC022F052
:1029B80030C023F0E1EC28F01EC02EF01EC0DFFF6F
:1029C800010E1FC0DBFF020E20C0DBFFFE0EDB5036
:1029D80026E1DFCF2EF0010EDBCF2FF0020EDBCF8A
:1029E80030F03034000E301807E6D8807F0E2E54B1
:1029F800000E2F54000E305401E28CD0D9CFE9FFDD
:102A0800DACFEAFF020ED880EB50FF0A06E6800E06
:102A1800EE5CFF0EEE58FF0EEF5801E27BD0FE0E83
:102A2800DB0424E1DFCF31F0010EDBCF32F0020E00
:102A3800DBCF33F03334000E331807E6D880FF0EAF
:102A48003154000E3254000E335464E3D9CFE9FFF9
:102A5800DACFEAFF020ED890EB50000A06E6000E25
:102A6800EE5C000EEE58000EEF5854E3020E346E82
:102A7800FE0EDB50345C24E1DFCF35F0010EDBCFF6
:102A880036F0020EDBCF37F03734000E371807E682
:102A9800D880FF0E35547F0E3654000E37543AE373
:102AA800D9CFE9FFDACFEAFF020ED880EB50FF0A50
:102AB80006E6000EEE5C800EEE58FF0EEF582AE395
:102AC800030E386EFE0EDB50385C27E1DFCF39F09D
:102AD800010EDBCF3AF0020EDBCF3BF03B34000EA9
:102AE8003B1807E6D880FF0E3954FF0E3A54000E03
:102AF8003B5410E3D9CFE9FFDACFEAFF020ED890B2
:102B0800EB50000A06E6000EEE5C000EEE58000ED2
:102B1800EF5803E20D8C010E27D0FE0EDB50030A9E
:102B280016E0010A14E0030A08E0050A06E0010AB3
:102B380004E0050A02E0040E17D0FC0EDBCFE9FF23
:102B4800FD0EDBCFEAFF000EDFCFEFFF0CD0FC0E4F
:102B5800DBCFE9FFFD0EDBCFEAFF000EDFCFEEFF94
:102B6800010EDBCFEDFF000E2E6E040EE15C02E2DB
:102B7800E16AE552E16E2E50E552E7CFD9FF120027
:102B8800D9CFE6FFE1CFD9FF020EE126FD0EDBCF5C
:102B9800E9FFFE0EDBCFEAFFEE6AEE6AEE6A010E8F
:102BA800DB6AFC0EDB50F36E010EDBCFF4FFF35053
:102BB800F45C53E20101E151EA6A000FE96E030E89
:102BC800EA22EFCFDFFF300EDF5C42E3DF50390847
:102BD8003FE3FD0EDBCFE9FFFE0EDBCFEAFFEECFD2
:102BE80031F0EECF32F0EFCF33F00A0E266E276ABF
:102BF800286A31C021F032C022F033C023F0E1EC62
:102C080028F0300EDF5C346E356A366A1E50342484
:102C18002E6E1F5035202F6E20503620306EFD0E40
:102C2800DBCFE9FFFE0EDBCFEAFF2EC0EEFF2FC0A1
:102C3800EEFF30C0EEFF0101E12BE1512E6E2F6A4D
:102C4800000E2E1807E1010E2F1804E1E16B02D0E7
:102C5800000E04D0010EDB2AA4D7010E2E6E020E40
:102C6800E15C02E2E16AE552E16E2E50E552E7CFFF
:102C7800D9FF12000650E66EE66A040E2E6E500E5C
:102C88002F6E306A2EC0E6FFE66E30C0E6FF64ECB9
:102C98002AF0316E050EE15E3150120000016051DC
:102CA80008E0010E2E6E6D50020B01E0010E2E5C45
:102CB8001BE10201CB07000ECC5BCD510BE1CB51E0
:102CC800CC1111E18B80D00ECB6F070ECC6F010EAB
:102CD800CD6F1200CB51CC114DE18B90D00ECB6F44
:102CE800070ECC6FCD6B1200600509E0020E605D27
:102CF80006E0040E605D03E0100E605D02E18B806B
:102D08001200200E605D36E10201CB07000ECC5B9D
:102D1800CD510AE1CB51CC112DE18B80100ECB6F38
:102D2800270ECC6F010E18D0CD050AE1CB51CC117E
:102D380021E18B90100ECB6F270ECC6F020E0CD0BA
:102D4800020ECD5D0BE1CB51CC1114E18B80A00EAE
:102D5800CB6F860ECC6F030ECD6F1200030ECD5DC8
:102D680009E3CB51CC1106E18B90100ECB6F270EE7
:102D7800CC6FCD6B120082A4010C000CD9CFE6FFFA
:102D8800E1CFD9FFE652A09A6A6A686A706A030EB0
:102D9800E66EE66AE66A710EE66E0F0EE66E17ECF0
:102DA8002AF02E6E050EE15E2E50160E6F6E9F0EE7
:102DB8006B6E7B0E696EDF6ADF502E6E2F6A100E07
:102DC8002E5C000E2F5810E2DF50040DF3CFE9FF00
:102DD800F4CFEAFF000EE926040EEA22EE6AEE6A54
:102DE800EE6AEE6ADF2AE8D76D8C6E6A6D986D9C84
:102DF80068A607D0689600017B6B806B816B826B3D
:102E0800F7D70001010E966F976F986B996B886BD7
:102E1800DF6A040EDF5C26E2EA6ADF34FE0BEA367C
:102E2800E96E6F0EE926000EEA22EE6AED6AEA6A9A
:102E3800DF34FE0BEA36E96E670EE926000EEA2259
:102E4800EE6AED6ADF50EA6A8C0FE96E000EEA223C
:102E5800EF6ADF50EA6A900FE96E000EEA22EF6A25
:102E6800DF2AD7D70001080E6F6F040E706F160E99
:102E7800706E0401400E026F040E036F400E016F66
:102E8800840E006F0001616B606BE552E552E7CF7D
:102E9800D9FF1200D9CFE6FFE1CFD9FFE6520001F2
:102EA800600507E16DBA05D0686A69806988020E15
:102EB800606F6850040B05E06950040B02E06894E9
:102EC800BFD86DB250D06850010B09E06950010BB2
:102ED80006E054DFA08A0001040E606F6890685015
:102EE800100B05E06950100B02E095D8689868ACA3
:102EF80012D069AC0FD0010EE66EE66A000EE66EDF
:102F0800E66A730EE66EE66A7DEC29F02E6E060E12
:102F1800E15E2E50689C6850200B04E06950200B3D
:102F280001E060D86850020B13E06950020B10E012
:102F3800010EE66EE66A000EE66EE66AE6687F0E49
:102F4800E66E7DEC29F02E6E060EE15E2E506A6A62
:102F5800040E0001E76E6019E8AE02D0E73402D033
:102F6800E750605D02E2A19A38D069A635D0DF6AE1
:102F7800040EDF5C31E268A62FD06CCF89F0000127
:102F88008951780BE842E842E8428A6F689689B529
:102F980006D08A51EA6A900FE96E000E05D08A5170
:102FA800EA6A8C0FE96E000EEA22EF708A5102E19C
:102FB8005ED810D0000EE66EE66A890EE66E000E48
:102FC800E66E720EE66EE66A7DEC29F02E6E060E4F
:102FD800E15E2E50DF2ACCD7A19AE552E552E7CF21
:102FE800D9FF120070A015D063C0E9FF64C0EAFFE2
:102FF800EF5080080DE16FC0E9FF70C0EAFFEF50A5
:10300800840806E163C0E9FF64C0EAFF8C0EEF6E36
:103018007090689A1200698468986D820001010EA8
:10302800886F000EE66EE66AE66EE66A750EE66E74
:10303800E66A7DEC29F02E6E060EE15E2E50120037
:103048000001886B000EE66EE66AE66EE66A740EAC
:10305800E66EE66A7DEC29F02E6E060EE15E2E50D5
:103068006D92699468A402D06894FCD71200D9CFF5
:10307800E6FFE1CFD9FFE652FD0E0001891553E1C5
:103088007E0E8915E8407F0B040DF3CF63F0F4CF73
:1030980064F0000E6327040E642363C065F064C007
:1030A80066F0657563C0E9FF64C0EAFFEF503C0B4A
:1030B800E842E8420D0835E1DF6A080EDF5C23E2EA
:1030C80063C0E9FF64C0EAFF020EE926000EEA22A7
:1030D800EE50EFCFEAFFE96EEF50E66EDF50EA6A96
:1030E800400FE96E040EEA22E552E750EF6E63C026
:1030F800E9FF64C0EAFF020EE926000EEA22EE2A82
:10310800EF22DF2ADAD763C0E9FF64C0EAFF020EC4
:10311800E926000EEA22400EEE6E040EED6E0DD882
:1031280007D03AD805D0FD0E8915040801E159D811
:10313800E552E552E7CFD9FF12000001776B956B96
:10314800986B996B8B6B786B6FC0E9FF70C0EAFF67
:10315800EF9E6F756FC0E9FF70C0EAFFEF9E6F7555
:1031680065C0E9FF66C0EAFFEF9E7B6B7C6B7D6BF9
:10317800806B816B826B8CD8000EE66EE66AE66E19
:10318800E66A030EE66EE66A7DEC29F02E6E060E00
:10319800E15E2E501BEF1CF0020E0001785D02E18B
:1031A800DBEF1CF0786B8B511AE165C0E9FF66C054
:1031B800EAFFEE52400EEF6E65C0E9FF66C0EAFF17
:1031C800020EE926000EEA22400EEE6E040EED6EA7
:1031D80065C0E9FF66C0EAFF8C0EEF6E12008B6BCC
:1031E8001200D9CFE6FFE1CFD9FFE6526FC0E9FF61
:1031F80070C0EAFFEF50400B01E0010EDF6E0001E6
:103208006F75080E605D08E142C46EFF6E5002E003
:10321800100E01D0040E606F780526E16FC0E9FF3B
:1032280070C0EAFF020EE926000EEA22480EEE6E92
:10323800040EED6E5DDB020E0001775D06E16FC0E6
:10324800E9FF70C0EAFF840E0DD0DF5006E16FC0C1
:10325800E9FF70C0EAFFC80E05D06FC0E9FF70C073
:10326800EAFF880EEF6E0FD080AF0CD08351841127
:1032780007E005D084C0FAFF00018351F96EFADF38
:103288000001809F786BE552E552E7CFD9FF120025
:1032980004014051600BE842E842E842E842E84253
:1032A800000901E0120041510C0A50E00B0A3FE00E
:1032B8000C0A31E0010A22E00B0A1EE0020A1CE0B7
:1032C800030A18E0080A10E0010A0CE00F0A08E0F7
:1032D800030A01E0120000017B8F080E606F1200E4
:1032E80064EF1BF07AEF1DF00001610E796F000E9C
:1032F8007A6F0CD0C1EF1BF0ABEF19F0445100010D
:10330800796F7A6B620E7927000E7A237B81010E22
:103318007C6F7B8F120000017B8F04014451EA6AA5
:10332800620FE96E000EEA2242C4EFFF1200000E9F
:10333800E66EE66AE66EE66A020EE66EE66A7DEC20
:1033480029F02E6E060EE15E2E5012001200D9CF23
:10335800E6FFE1CFD9FF030EE1260401420510E1A3
:1033680040511F0B00090CE100017B8F030E040183
:10337800415D04E10001010E876F02D00001876BF7
:103388000401425101E003D140511F0B020801E042
:10339800FED044510F0B000901E1F9D044510F0B45
:1033A800030801E2F4D0200E0001605D01E0EFD0D7
:1033B8007B8F040144BF16D044510F0BE96EEA6AB3
:1033C800D890E936EA36670EE926000EEA22EECFF3
:1033D800DEFFEDCFDDFF44510F0BEA6A900FE96E77
:1033E800000E15D044510F0BE96EEA6AD890E93601
:1033F800EA366F0EE926000EEA22EECFDEFFEDCFA9
:10340800DDFF44510F0BEA6A8C0FE96E000EEA22C9
:10341800020EEFCFDBFFD950020FE96EDACFEAFFD9
:10342800EF50010B03E1000EDF9401D0DF8444BFAD
:103438000BD044510F0BE96EEA6AD890E936EA36A8
:10344800670EE926000E0AD044510F0BE96EEA6AAE
:10345800D890E936EA366F0EE926000EEA22DECF6A
:10346800EEFFDDCFEDFF030E415D20E1DECFE9FF8A
:10347800DDCFEAFFEF50800B11E044BF07D0445185
:103488000F0BEA6A900FE96E000E06D044510F0B3D
:10349800EA6A8C0FE96E000EEA22EF82840EDECF14
:1034A800E9FFDDCFEAFFE850EF1271D0DF74DECF1D
:1034B800E9FFDDCFEAFFEF50800B1BE0DECFE9FF2D
:1034C800DDCFEAFFEF9EDECFE9FFDDCFEAFFEF8C2D
:1034D800020EE66EE66ADECFE6FFDDCFE6FF050EFA
:1034E800E66EE66A7DEC29F02E6E060EE15E2E5041
:1034F80005D0DECFE9FFDDCFEAFFEF8CDF74D950CE
:10350800020FE96EDACFEAFFEF50020B0EE1DECFD1
:10351800E9FFDDCFEAFFEF50800B32E0DECFE9FFB5
:10352800DDCFEAFFEF50040B2BE1040144BF07D0C5
:1035380044510F0BEA6A900FE96E000E06D0445111
:103548000F0BEA6A8C0FE96E000EEA22EF923B0E2F
:103558002E6EDECFE9FFDDCFEAFFE850EF16020E50
:10356800E66EE66ADECFE6FFDDCFE6FF050EE66E25
:10357800E66A7DEC29F02E6E060EE15E2E5007D02D
:103588003B0EDECFE9FFDDCFEAFFE850EF16030E72
:10359800E15C02E2E16AE552E16EE552E7CFD9FF6C
:1035A8001200000196514DE1010E966F975149E1C5
:1035B800010E976F020E785D0DE16FC0E9FF70C0D4
:1035C800EAFFEE52EF6A6FC0E9FF70C0EAFFC80E6B
:1035D800EF6E1200780535E18B6B63C0E9FF64C0BC
:1035E800EAFFEE52400EEF6E63C0E9FF64C0EAFFE7
:1035F800020EE926000EEA22400EEE6E040EED6E73
:1036080063C0E9FF64C0EAFF840EEF6E010E8B6FA2
:1036180065C0E9FF66C0EAFFEE52400EEF6E65C076
:10362800E9FF66C0EAFF020EE926000EEA22400E14
:10363800EE6E040EED6E65C0E9FF66C0EAFF800E0F
:10364800EF6E12000001986B996B020E785D18E11D
:1036580065C0E9FF66C0EAFFEE52400EEF6E65C036
:10366800E9FF66C0EAFF020EE926000EEA22480ECC
:10367800EE6E040EED6E65C0E9FF66C0EAFF1DD070
:103688007C510401465D00017D510401475904E263
:1036980046C47CF047C47DF02BD96FC0E9FF70C0E9
:1036A800EAFF020EE926000EEA22480EEE6E040E2C
:1036B800ED6E6FC0E9FF70C0EAFFC80EEF6E120032
:1036C800800E0401405D58E10001C00E7B6F0401CB
:1036D8004351030A2FE0010A09E0030A4BE1000104
:1036E800E40E796F550E7A6F120E3ED04251F66E87
:1036F800F76AD890F636F7365D0EF626560EF7229C
:103708000900F5CF79F00A00F5CF7AF0020E000132
:10371800F76A7925F66E7A51F7220800F5CF7CF022
:10372800030EF76A7925F66E7A51F7220800F5CF6D
:103738007DF01200030E425D1AE24251F66EF76AFE
:10374800D890F636F7365F0EF626560EF7220900A1
:10375800F5CF79F00A00F5CF7AF079C0F6FF7AC094
:10376800F7FF0800F55000017C6F7D6B1200000127
:103778007B6B120000017B6B1200D9CFE6FFE1CF13
:10378800D9FF020EE1260401486B496B40511F0B1B
:10379800020A11E0030A0CE0010A35E100017B8FFF
:1037A80004014881000187052EE1040148832BD0DC
:1037B80000017B8F28D000017B8F040144BF0BD010
:1037C80044510F0BE96EEA6AD890E936EA36670E7B
:1037D800E926000E0AD044510F0BE96EEA6AD89028
:1037E800E936EA366F0EE926000EEA22EECFDEFF52
:1037F800EDCFDDFFDECFE9FFDDCFEAFFEF50040BB1
:1038080002E0010E486F00017BAF07D0480E796FC8
:10381800040E7A6F7B81020E7C6F020EE15C02E27D
:10382800E16AE552E16EE552E7CFD9FF12006D98E3
:1038380000017BBF2BD080AF09D0020E786F995161
:1038480001E100DF0001976B966B120065C0E9FF8C
:1038580066C0EAFFEE52400EEF6E65C0E9FF66C033
:10386800EAFF020EE926000EEA22400EEE6E040E72
:10387800ED6E65C0E9FF66C0EAFF8C0EEF6E6FC0A3
:10388800E9FF70C0EAFF840EEF6E1200040140AF3A
:103898000DD00001010E786F985101E1D3DE0001CF
:1038A800976B966B955123E1D5EF1AF00001020E44
:1038B800786F65C0E9FF66C0EAFFEE52400EEF6E12
:1038C80065C0E9FF66C0EAFF020EE926000EEA229B
:1038D800400EEE6E040EED6E65C0E9FF66C0EAFFAD
:1038E800840EEF6E976B966B955101E15ADE1200CC
:1038F800D9CFE6FFE1CFD9FFE652400EDF6E0001D7
:103908007C5D000E7D590AE27CC0DFFF775102E141
:10391800010E03D0770502E1020E776FDF502F6AA0
:10392800E8507C5D7C6F2F507D597D6F6FC0E9FF3B
:1039380070C0EAFFEE52DFCFEFFF480E856F040E2E
:10394800866F7BB118D0DF502DE079C0F6FF7AC0C2
:10395800F7FF792B000E7A230800F550E66E85C034
:10396800E9FF86C0EAFF852B000E8623E552E75063
:10397800EF6EDF06E8D7DF5015E079C0E9FF7AC0BF
:10398800EAFF792B000E7A23EF50E66E85C0E9FF37
:1039980086C0EAFF852B000E8623E552E750EF6EBE
:1039A800DF06E9D7E552E552E7CFD9FF1200D9CFB4
:1039B800E6FFE1CFD9FF020EE12663C0E9FF64C04C
:1039C800EAFFEE52EFCFDFFFDFCF2EF02E500001DF
:1039D800815D000E825902E281C0DFFFDF502E6E4A
:1039E8002F6AE850815D816F2F508259826F010ED6
:1039F800DB6ADF50F36E010EDBCFF4FFF350F45CAB
:103A080016E2010EDB50EA6A480FE96E040EEA225C
:103A1800EF50E66E7EC0E9FF7FC0EAFF7E2B000E06
:103A28007F23E552E750EF6E010EDB2AE2D7000E46
:103A3800D8808155000E825527E265C0E9FF66C02F
:103A4800EAFFEE52400EEF6E65C0E9FF66C0EAFF7E
:103A5800020EE926000EEA22480EEE6E040EED6E06
:103A680063C0E9FF64C0EAFFEF50400B06E165C0A0
:103A7800E9FF66C0EAFFC80E05D065C0E9FF66C069
:103A8800EAFF880EEF6E28D065C0E9FF66C0EAFF3E
:103A9800EE52400EEF6E65C0E9FF66C0EAFF020E07
:103AA800E926000EEA22400EEE6E040EED6E65C0A9
:103AB800E9FF66C0EAFF840EEF6E8351841107E0C8
:103AC80005D084C0FAFF00018351F96EFADF0001C6
:103AD800809F955101E165DD020EE15C02E2E16A39
:103AE800E552E16EE552E7CFD9FF1200D9CFE6FFE4
:103AF800E1CFD9FFE65200017B8F030EE66EE66A3E
:103B0800E66A710EE66E0F0EE66E17EC2AF02E6E60
:103B1800050EE15E2E50DF6ADF502E6E2F6A100E02
:103B28002E5C000E2F5810E2DF50040DF3CFE9FF92
:103B3800F4CFEAFF000EE926040EEA22EE6AEE6AE6
:103B4800EE6AEE6ADF2AE8D76D8C010EE66EE66A49
:103B5800E66A620EE66E000EE66E17EC2AF02E6E2E
:103B6800050EE15E2E506D9C0001080E6F6F040E6D
:103B7800706F000E636F040E646F63C065F0666F4C
:103B880042C461F0615102E1100E12D0010EE66EDE
:103B9800E66A610EE66E000EE66E010EE66EE66AF5
:103BA8007DEC29F02E6E060EE15E2E500001200EEF
:103BB800606FE552E552E7CFD9FF1200D9CFE6FF93
:103BC800E1CFD9FF020EE126000EDE6E040EDD6E97
:103BD800FD0EDB50E824306EFE0EDB50040DF35072
:103BE8003024040DF4CF2FF0D9CFE9FFDACFEAFF64
:103BF800F350EE262F50ED22DECFE9FFDDCFEAFFAE
:103C0800EF9EFD0EDB500AE1FE0EEA6ADB34FE0B86
:103C1800EA36E96E670EE926000E09D0FE0EEA6A5A
:103C2800DB34FE0BEA36E96E6F0EE926000EEA2257
:103C3800DECFEEFFDDCFEDFFDECFE9FFDDCFEAFF20
:103C4800EF9CDECFE9FFDDCFEAFF040EE926000E88
:103C5800EA22EF8C020EE15C02E2E16AE552E16ED3
:103C6800E552E7CFD9FF1200D9CFE6FFE1CFD9FF60
:103C7800020EE126FD0EDBA407D0E66AFE0EDBCFBE
:103C8800E6FF9CDFE552E552FD0EDBA208D0010EEF
:103C9800E66EFE0EDBCFE6FF91DFE552E552FE0E43
:103CA800DB502F6A700F2E6E0F0E2F222EC0DEFFF4
:103CB8002FC0DDFFDECFE9FFDDCFEAFFFD0EDBCF52
:103CC800EFFF020EE15C02E2E16AE552E16EE552C5
:103CD800E7CFD9FF1200D9CFE6FFE1CFD9FF020E17
:103CE800E126FE0EDB5020E165C0E9FF66C0EAFF71
:103CF800EE52400EEF6E65C0E9FF66C0EAFF020EA5
:103D0800E926000EEA22400EEE6E040EED6E65C046
:103D1800E9FF66C0EAFF8C0EEF6E6FC0E9FF70C066
:103D2800EAFF840EEF6E3BD0FD0EDB50E824306EC8
:103D3800FE0EDB50040DF3503024040DF3CF2EF0AB
:103D4800F4CF2FF0000E2E26040E2F222EC0DEFFF9
:103D58002FC0DDFF840EDECFE9FFDDCFEAFFE8509C
:103D6800EF12FD0EDB50E824306EFE0EDB50040D22
:103D7800F3503024010F040DF3CF2EF0F4CF2FF0C1
:103D8800000E2E26040E2F222EC0DEFF2FC0DDFFD0
:103D9800840EDECFE9FFDDCFEAFFE850EF12020E16
:103DA800E15C02E2E16AE552E16EE552E7CFD9FF54
:103DB8001200D9CFE6FFE1CFD9FF020EE126FD0EB2
:103DC800DB500AE0FE0EEA6ADB34FE0BEA36E96EE7
:103DD8006F0EE926000E09D0FE0EEA6ADB34FE0BF0
:103DE800EA36E96E670EE926000EEA22EECFDEFF1C
:103DF800EDCFDDFFD9CFE9FFDACFEAFFEE50ED10C6
:103E080003E1F36AF46A44D0DECFE9FFDDCFEAFFCD
:103E1800020EE926000EEA22FB0EDBCFEEFFFC0EB7
:103E2800DBCFEDFFDECFE9FFDDCFEAFFEE52FA0E82
:103E3800DBCFEFFF400EDECFE9FFDDCFEAFFE85032
:103E4800EF16880EDECFE9FFDDCFEAFFE850EF126C
:103E5800FD0EDB500AE0FE0EEA6ADB34FE0BEA36A2
:103E6800E96E6F0EE926000E09D0FE0EEA6ADB3411
:103E7800FE0BEA36E96E670EE926000EEA22EF74B9
:103E8800DECF2EF0DDCF2FF02EC0F3FF2FC0F4FFD2
:103E9800020EE15C02E2E16AE552E16EE552E7CF2B
:103EA800D9FF1200D9CFE6FFE1CFD9FF6DA84ED0D8
:103EB800FE0EEA6ADB34FE0BEA36E96E6F0EE9267F
:103EC800000EEA22EE50EFCFEAFFE96E400EEE1642
:103ED800EE6AEE6AEE6AFE0EEA6ADB34FE0BEA363A
:103EE800E96E6F0EE926000EEA22EE50EFCFEAFFE8
:103EF800E96EEE7CFE0EEA6ADB34FE0BEA36E96E0A
:103F08006F0EE926000EEA22EF74400E2E6EFE0EAA
:103F1800EA6ADB34FE0BEA36E96E6F0EE926000E1C
:103F2800EA22EE50EFCFEAFFE96E2E50EF16FE0EB2
:103F3800EA6ADB34FE0BEA36E96E6F0EE926000EFC
:103F4800EA22EE50EFCFEAFFE96EEF7CE552E7CFC9
:103F5800D9FF12006D6A696A0001606B12000001E6
:103F6800605113E16D6A696A160E6F6E9F0E6B6E73
:103F78007B0E696ED08EA29AA08AF28E6DB602D0A0
:103F88006D86FCD70001010E606F120006EC25F06B
:103F9800FB0EDBCFF3FFDB06F35000090AE054EC1D
:103FA80025F0FA0EBFEC25F0F3E12F1CF1E1010E2C
:103FB80001D0000E35EF25F006EC25F03B0EE1248C
:103FC80002E3E168E652E16E010EDB6A020EDB6A8B
:103FD800F90EDBCFF6FFFA0EDBCFF7FFFB0EDBCFD8
:103FE800F8FF0800F550DF6EDF5002E159EF24F0CA
:103FF800250EDF5C02E04CEF24F0030EDB6A040EB2
:10400800DB6A050EDB6A060EDB6A070EDB6A6EECFE
:1040180024F02D0EDF5C0CE02B0EDF5C09E0200E97
:10402800DF5C06E0230EDF5C03E0300EDF5C1AE1A4
:10403800DF50300A14E0130A0FE0030A0AE00B0A03
:1040480005E0060AE4E1030EDB80E1D7030EDB821C
:10405800DED7030EDB84DBD7030EDB86D8D7030E4F
:10406800DB88D5D72A0EDF5C1BE16AEC24F0B8ECBC
:1040780024F010E0030EDB8022682368130EDBCFE8
:1040880027F0140EDBCF28F02AEC29F0040E20C00C
:10409800DBFF03D0130EA1EC24F06EEC24F00BD060
:1040A800090EDB6A0FEC25F003E083EC25F0FAD764
:1040B800090EA1EC24F0030EDBB0DB982E0EDF5CBA
:1040C8001BE16EEC24F02A0EDF5C0BE16AEC24F0B5
:1040D800B8EC24F003E1130EF3EC24F06EEC24F0BA
:1040E8000BD0090EDB6A0FEC25F003E083EC25F01A
:1040F800FAD7090EF3EC24F0680EDF5C07E16EECEA
:1041080024F0680EDF5C1DE1030E18D0740EDF5C2E
:1041180017E07A0EDF5C14E0480EDF5C06E0540E10
:10412800DF5C03E05A0EDF5C02E1020E07D06C0E82
:10413800DF5C03E06A0EDF5C04E1010E46EC25F06B
:10414800C9DBDF506E0A01E17FD31E0A01E192D17B
:10415800200A01E18FD13F0A01E149D11A0A01E1A0
:1041680046D10D0A01E143D1200A01E140D13A0AC2
:1041780001E13DD1200A01E13AD1260A01E135D118
:104188000D0A01E132D11A0A01E1D9D0200A4AE028
:10419800300A1FE0460A0EE0250A01E083D3D95011
:1041A800F90FE96EFF0EDA20EA6E010EEE5E000EE0
:1041B800EE5AEE5A54EC25F0250EE66E95DB03E137
:1041C8002F1C01E169D350EC25F001E26BD3DB2A07
:1041D80069D3080EDB6A040EDB50010806E2040E00
:1041E800DB0418EC25F0DB508BDB080EDB5009E014
:1041F800030EDB50010B05E172DB01E04DD3080E25
:10420800DB6A64DBEFCFDFFFC8EC25F003E12F1C8E
:1042180001E142D350EC25F001E3DB2A60DB01E148
:1042280041D33AD3070EDB5002080FE194EC25F096
:10423800030E5BEC25F00E0EEECFDBFF0F0EEECF7C
:10424800DBFF100EEECFDBFF20D0F70EDBCF31F017
:10425800F80EDBCF32F0020E315E000E325AF70E46
:1042680031C0DBFFF80E32C0DBFF31C0E9FF32C0DE
:10427800EAFF4BEC25F0306A0E0E2EC0DBFF0F0E66
:104288002FC0DBFF100E30C0DBFF0E0EDBCFE6FFCA
:104298000F0EDBCFE6FF100EDBCFE6FF3FEC2AF078
:1042A800E552E552E552130E21C0DBFF140E22C081
:1042B800DBFF060EDB5005E0130E8FEC25F001E264
:1042C8006ADBB3EC25F002E2130E37DB76EC25F05F
:1042D80006E0040E8FEC25F002E2050E2EDB030E3D
:1042E800DBB005D0FCDA01E0D7D2080EDB6A090E94
:1042F800DB6A0E0EDBCFF6FF0F0EDBCFF7FF100EDB
:10430800DBCFF8FF0800F550DF6EDF5014E0B9ECA2
:1043180025F011E2C8EC25F003E12F1C01E1BCD225
:10432800BBDB01E3DB2A090EDB2AD9500E0FE96E4D
:10433800000ECBDBE7D7D3DA01E1B4D2ADD2C6DACF
:10434800110EEECFDBFF120EEDCFDBFF110EDBCF30
:10435800E6FF120EDBCFE6FF31EC2AF0E552E5521C
:10436800130EF3CFDBFF140EF4CFDBFF060EDB508A
:1043780004E0130ED0DB01E20EDBB3EC25F002E221
:10438800130EDBDAAFDB05E0040EC5DB02E2050E37
:10439800D4DA030EDBB005D0A2DA01E07DD2080E34
:1043A800DB6A090EDB6A110EDBCFE9FF120EDBCFE9
:1043B800EAFFEFCFDFFFDF5014E0D7DB12E2E4DBE8
:1043C80003E12F1C01E168D267DB01E3DB2A090E58
:1043D800DB2A110EDB2ADBCFE9FF120EE8E3DB2A2A
:1043E800E6D77DDA01E15ED257D2030EDB8E070EE7
:1043F800DB0410E195DB040E5ADB0A0EEECFDBFF7F
:104408000B0EEECFDBFF0C0EEECFDBFF0D0EEECF6B
:10441800DBFF6CD0070EDB5003082CE1030EDBAE8C
:104428000DD0B2DA020E76DAEFCF2EF02F6A306AAC
:10443800316A2EAE39D02F68306835D0F70EDBCF11
:104448002FF0F80EDBCF30F0020E2F5E000E305A40
:10445800F70E2FC0DBFFF80E30C0DBFF2FC0E9FFDF
:1044680030C0EAFFEFCF2EF00A0E2EC0DBFF0B0E96
:10447800DB6A38D0070EDB50020809E1030EDBAE19
:1044880004D059DB30AE10D00ED055DB0DD0030E62
:10449800DBAE12D079DA020E3DDAF9DA306A316A27
:1044A8002FAE02D030683168E2DA0C0E30C0DBFF84
:1044B8000D0E31C0DBFF1AD0F70EDBCF30F0F80E4F
:1044C800DBCF31F0020E305E000E315AF70E30C0ED
:1044D800DBFFF80E31C0DBFF30C0E9FF31C0EAFF77
:1044E800D6DAC5DA0C0EDB6A0D0EDB6A060EDB5077
:1044F80005E1010EF36E050EF3CFDBFF150EDB6A47
:10450800160EDB6AD950370F2E6E000EDA202F6E8A
:10451800390E2EC0DBFF3A0E2FC0DBFF380EDB6AE8
:10452800080EDB6A0A0EAEDADF50780A12E0200ABB
:1045380010E0280A0CE0200A0AE03F0A06E00D0A0B
:1045480002E0200A08E1020E05D0080E03D0080E8A
:10455800DF26100E97DA030EDBBE02D0DB92DB9467
:10456800DB50800B24E08ADAD890030EEB50000A67
:1045780008E6000EEE5C000EEE58000EEE58000E37
:10458800EE5815E213DA256826682768286833ECA0
:104598002BF00A0E1CC0DBFF0B0E1DC0DBFF0C0E40
:1045A8001EC0DBFF0D0E1FC0DBFF2D0E08D0030E53
:1045B800DBA202D02B0E03D0DBA408D0200EF36EB2
:1045C800170EF3CFDBFF150EDB2A02D0170EDB6ABE
:1045D800050EDB5003E1B7D901E189D0FA0E2E6E42
:1045E800570E2F6E000E306E070EDBCF31F0326A99
:1045F800336A346A31C025F032C026F033C027F060
:1046080034C028F0D3D991EC2BF02E501C24F36E33
:104618002F501D20F46E30501E20F86EF4CFF7FF97
:10462800F3CFF6FF0800090EF5CFDBFF580EDF5C6D
:104638000FE1610EF36E090E7BD90AE3200E2E6E90
:10464800090EDBCFE7FF2E50E75E090EE7CFDBFF51
:10465800070EDBCF2EF02F6A306A316A0FDA2EC0D0
:1046680025F02FC026F030C027F031C028F0EECF5B
:1046780020F0EECF21F0EECF22F0EFCF23F091EC37
:104688002BF023C0EDFF22C0EDFF21C0EDFF20C0BD
:10469800EFFF390EDBCFE9FFDB063A0EDBCFEAFF8F
:1046A80001E2DB06090EDBCFEFFF150EDB2A4BD943
:1046B80095E1030EDBA61DD06F0EDF5C06E1C1D9C4
:1046C80018E3150EDB285BDA14D0780EDF5C09E0FE
:1046D800580EDF5C06E0620EDF5C03E0420EDF5C32
:1046E80008E1020EF36E160EF3CFDBFF02D0150EB3
:1046F800DB6A030EDB50100B0EE0040EDBCF2EF04E
:10470800050EDB50D8802E5406E2060EDB5003E17E
:10471800040EDB5034DA95D90AE2050EDBCFE7FF49
:10472800150EDB50E75E050EE7CFDBFF02D0050E66
:10473800DB6A040EDBCF2EF0160E45D9D8802E5436
:1047480014E2160EDBCFE6FF150EDBCFE6FF040EF4
:10475800DBCFE6FF050EDB50E552E75CE552D8807B
:10476800E754E552D880E7545FD9030EDB50010BBC
:104778000BE1080EDB5008E0B2D801E08DD0080E3E
:10478800DB50BED8080EDB6A170EDB5007E088D96D
:10479800170EF1D903E12F1C01E17ED0160EDB5074
:1047A80016E07ED9300EE66E9FD802E12F1C74E029
:1047B80077D9DFCFE6FFB0EC2AF0E552E552E552B3
:1047C800F4CF2FF00001F31C02E12F1C65E0050E69
:1047D800DBCF2EF0160EDB50D8802E5409E2050EE2
:1047E800DBCFE7FF160EDB50E75E050EE7CFDBFFFA
:1047F800300EE66E050ECBD94FE1390EDB2ADBCF42
:10480800E9FF3A0E01E3DB2ADBCFEAFF090EEFCF1F
:10481800DBFFDB500EE044D9090EADD902E12F1CB5
:104828003BE0390EDB2ADBCFE9FF3A0EEDE3DB2A6A
:10483800EBD755D831E1160EDBCFE6FF080EC3D80B
:10484800E552E7245DD82ED0070EDB50030A1CE0A2
:10485800010A14E0030A07E07BD9DBCFEEFF020E62
:10486800DBCFEDFF1FD0F5D8336A31AE02D0326806
:1048780033682CD8BCD833C0EEFF14D0EAD831BE88
:10488800326824D8B4D80ED063D9DBCFEFFF0AD072
:104898007BD905E12F1C03E1F368F46810D0FCD83C
:1048A80001E3DB2A79D9F5EF1FF0010EDBCF2EF0FB
:1048B800020EDBCF2FF02EC0F3FF2FC0F4FF3B0E0C
:1048C800E15C02E2E16AE552E16ECBD029D9020E41
:1048D8005BEF25F061D90800F550DF6E1200200E5D
:1048E800E66E080ECBEF25F0B0EC2AF0E552E55263
:1048F800E552F3CF2EF0F4CF2FF00001F31C120095
:104908002E6E2F6AD950010F4DD92E50EE262F50FA
:10491800ED221200325E000E335AF70E32C0DBFF72
:10492800F80E33C0DBFF32C0E9FF33C0EAFF1200E4
:10493800DBCFF4FFF350F45C1200DB50E76E040E9B
:10494800E7CFDBFF12000A0EDBCF2EF00B0EDBCF1A
:104958002FF00C0EDBCF30F00D0EDBCF31F02E50E8
:104968002F10301031101200130EEECFDBFF140E93
:10497800EDCFDBFF130EDBCF2EF0140EDBCF2FF0C5
:104988000001800E2F141200F70EDBCF32F0F80E64
:10499800DBCF33F01200050EDB50E66ED950130F53
:1049A80001D9E552E750EE6EED6A12000A0EDBCF30
:1049B80020F00B0EDBCF21F00C0EDBCF22F00D0E1A
:1049C800DBCF23F01200DBCFE6FF150EDBCFE6FFCF
:1049D800050EDB50E552E724E552E7241200DB50D0
:1049E800CED8010EF36E060EF3CFDBFF1200EE50A9
:1049F800EFCFEAFFE96E30C0EEFF31C0EEFF32C004
:104A0800EEFF1200D9CFE6FFDACFE6FFE1CFD9FFFC
:104A1800E2CFDAFF1200DFCFE6FFE66A7FEC2BF089
:104A2800E552E552F3501200E76E080EE7CFDBFFC0
:104A38001200EECF2EF0EECF2FF0EFCF30F0316A2C
:104A48001200050EDBCF2EF0150EDB50D8802E5449
:104A58001200010EDBCF30F0020EDBCF31F0326AEC
:104A68001200E552E5CFDAFFE7CFD9FF12000A0EB0
:104A78002EC0DBFF0B0E2FC0DBFF1200D9500A0F30
:104A8800D6EF25F0F36E070EF3CFDBFF1200EECF63
:104A98002EF0EFCF2FF01200010EDB2A020E1200CB
:104AA800FC0EDBCFE6FFFD0EDBCFE6FF12002E5E2D
:104AB800000E2F5AF70E2EC0DBFFF80E2FC0DBFFBB
:104AC8002EC0E9FF2FC0EAFF1200DA20EA6EEF2AB3
:104AD800EECFF6FF000EEF22EECFF7FFEF22EECF7C
:104AE800F8FF1200040EDBCFE6FF130EDB50E55291
:104AF800E75C9ADFDB5004DF060EDB501200090E7C
:104B0800DB500A0DF350DF24D00FE76E090EE7CF14
:104B1800DBFF6EEF24F0DB50F36E050E9CEF24F004
:104B2800F70EDBCF2EF0F80EDBCF2FF01200DFCF21
:104B3800E6FF78EF24F028DF030EECDE1DEF25F00A
:104B4800CAEC1FF0E552E552E552E55200091200A1
:104B5800BDDEEE50EFCFEAFFE96E010E1200130E34
:104B6800DB50F36E040E9CEF24F0040EDB50F36E62
:104B7800090E9CEF24F0DBCFE6FF78EF24F0E76E18
:104B8800050EE7CFDBFF12008BDF9BEF25F0DBCFB5
:104B9800E6FF86DFA4EF25F0D950F90FE96EFF0E86
:104BA80069EF25F0E96E000EDA20EA6E12000401C2
:104BB80040511F0B010801E012004051600BE84210
:104BC800E842E842E842E842010801E012004451A4
:104BD80003E0440501E012004151220A31E0030AD2
:104BE80024E0010A15E0210A0DE0010A01E01200A3
:104BF8000001DF0E796F020E7A6F080E7C6F7D6BF5
:104C08007B8121D00001DF0E796F020E7A6F1BD0F5
:104C180046C481F047C482F00001880E7E6F050EFD
:104C28007F6F836B846B808F12000001880E796F11
:104C3800050E7A6F070E7C6F7D6BC10E7B6F1200BD
:104C480042C4DAF200017B8F12000501886B4B0E1B
:104C5800896F8A6B8B6B8C6B8D6B080E8E6F020164
:104C6800CE6B1A0EE66E020EE66E38EC1EF0E552BA
:104C7800E5521E0EE66E030EE66E38EC1EF0E552A7
:104C8800E552400EE66E080EE66E050EE66EE66A22
:104C9800030EE66EDDEC1EF02E6E050EE15E2E5064
:104CA800F3CFD6F2F4CFD7F20201D86BD96BCF6B22
:104CB8001200D9CFE6FFE1CFD9FF0201CE6BD65162
:104CC800D71102E1000E08D0D6C2E9FFD7C2EAFF29
:104CD800EF50800B01E0010E000945E1FC0EDBCF2F
:104CE8002EF0D6C2E9FFD7C2EAFFEE52EF50D880C5
:104CF8002E5408E2D6C2E9FFD7C2EAFFEE52FC0EF4
:104D0800EFCFDBFFCE6BFC0EDB50CE5D19E2CE5150
:104D1800EA6A080FE96E050EEA22EF50E66ECE51F8
:104D2800E76EFD0EDBCFE9FFFE0EDBCFEAFFE750B3
:104D3800E926000EEA22E552E750EF6ECE2BE3D7C4
:104D4800400EE66E080EE66E050EE66EE66A030E87
:104D5800E66EDDEC1EF02E6E050EE15E2E50F3CFF2
:104D6800D6F2F4CFD7F20201CE51E552E7CFD9FF00
:104D78001200D9CFE6FFE1CFD9FFA09A0201CF51A7
:104D88000CE1FD0EDBCFD0F2FE0EDBCFD1F2FC0E34
:104D9800DBCFD4F2010ED56FCF6FA08AE552E7CFF3
:104DA800D9FF1200D9CFE6FFE1CFD9FF030EE126E4
:104DB800A09A0201CF512DE1DF6AFD0EDBCF22F070
:104DC800FE0EDBCF23F0DE5222C0DEFF23C0DDFF64
:104DD800DD52DF2ADF502E6E2F6AFF0E2E1802E1F9
:104DE8002F500BE0010EDBCFE9FFDB2A020EDBCFF1
:104DF800EAFF01E3DB2AEF50ECE1FD0EDBCFD0F256
:104E0800FE0EDBCFD1F2DFCFD4F20201010ED56F57
:104E1800CF6FA08A030EE15C02E2E16AE552E16E1F
:104E2800E552E7CFD9FF1200D9CFE6FFE1CFD9FF8E
:104E3800030EE126A09A0201CF512EE1DF6AFD0E92
:104E4800DBCF22F0FE0EDBCF23F0DE5222C0DEFFE6
:104E580023C0DDFFDD52DF2ADF502E6E2F6AFF0EE2
:104E68002E1802E12F500CE0010EDBCFF6FFDB2AF3
:104E7800020EDBCFF7FF01E3DB2A0800F550EBE178
:104E8800FD0EDBCFD0F2FE0EDBCFD1F2DFCFD4F2B6
:104E98000201D56B010ECF6FA08A030EE15C02E21E
:104EA800E16AE552E16EE552E7CFD9FF1200D9CFAA
:104EB800E6FFE1CFD9FF020EE126A09A0201D85100
:104EC800D91102E1000E08D0D8C2E9FFD9C2EAFF21
:104ED800EF50800B01E0010E000906E1030ECF5DE3
:104EE80001E1CF6BCF5102E1A08A7ED0020ECF5DE7
:104EF80016E1E66A000EE66EE66A010EE66E030E3D
:104F0800E66EDDEC1EF02E6E050EE15E2E50F3CF40
:104F1800D8F2F4CFD9F20201030ECF6F64D0CF05D7
:104F280062E1400E2E6E2F6AD4512E5C000E2F586F
:104F380003E2400EDF6E02D0D4C2DFFFDF50D45D43
:104F4800D46F480ED26F050ED36F010EDFCFDBFF93
:104F5800D55116E1010EDB5028E0D0C2F6FFD1C2D0
:104F6800F7FF0800F550D2C2E9FFD3C2EAFFEF6E9F
:104F7800D22B000ED323D02BD123010EDB06EAD788
:104F8800010EDB5012E0D0C2E9FFD1C2EAFFEF50B8
:104F9800D2C2E9FFD3C2EAFFEF6ED22B000ED323B1
:104FA800D02BD123010EDB06EBD70201D45107E148
:104FB800400EDF5C02E1020E01D0030ECF6FDFCF9F
:104FC800E6FF480EE66E050EE66E010EE66E030E6F
:104FD800E66EDDEC1EF02E6E050EE15E2E50F3CF70
:104FE800D8F2F4CFD9F2A08A020EE15C02E2E16ABB
:104FF800E552E16EE552E7CFD9FF120053746174B0
:1050080075733D25690D0A002135204572723A20D5
:105018004E65656420636F6D6D61206E6578742CD4
:1050280020666F756E643A20272563270D0A0050A5
:10503800492C2531750D0A004D522C253033750D3C
:105048000A002C25303475004100492C253033697D
:105058002C253033692C253033690D0A002138207E
:105068004572723A20556E6B6E6F776E20636F6D66
:105078006D616E642027256325633A2532582532F1
:1050880058270D0A002138204572723A20556E6B58
:105098006E6F776E20636F6D6D616E642027256378
:1050A8003A253258270D0A002137204572723A20D6
:1050B8004578747261207061726D617465720D0A51
:1050C800002136204572723A20496E76616C696417
:1050D80020706172616D7465722076616C75650D02
:1050E8000A002134204572723A204D697373696E43
:1050F8006720706172616D657465722873290D0A85
:10510800002133204572723A205258204275666653
:105118006572206F76657272756E0D0A00213220F5
:105128004572723A20545820427566666572206F3F
:1051380076657272756E0D0A002130200D0A002006
:1051480008002573001B5B421B5B314B1B5B304720
:015158000056
:10515A001A6AE86A28AEBAEF28F0256C261E271EBE
:10516A00281E2622272228221A1E23AEC5EF28F03F
:10517A00206C211E221E231E2122222223221A1ED5
:10518A0091EC2BF023BEDCEF28F01AAE000C206C59
:10519A00211E221E231EE86A2122222223221C6C9F
:1051AA001D1E1E1E1F1E1D221E221F22000C1ABE9D
:1051BA00CCEF28F01B88FF0C23C02DF022C02CF066
:1051CA0021C02BF021502602F4CF1FF0F3CF1EF09E
:1051DA0022502702F4CF21F0F3CF20F02602F35019
:1051EA001F26F4502022E86A21222B502702F3506E
:1051FA001F26F4502022E86A212223502602F35067
:10520A002026F450212223502702226AE86A222209
:10521A00F3502126F45022222B502802F350202644
:10522A00F4502122236AE86A222223222C502802DF
:10523A00F3502126F4502222E86A23222D50280214
:10524A00F3502226F4502322000C23C02DF022C052
:10525A002CF022502702F4CF21F0F3CF20F0235074
:10526A002802F4CF23F0F3CF22F02702F3502126AD
:10527A00F4502222E86A23222C502802F3502126D5
:10528A00F4502222E86A232228AE50EF29F02C504B
:10529A00225E2D50235A2DAE000C2750225E285034
:1052AA00235A000C08D80001605102E1B3EC1FF048
:1052BA00C0EC06F0F8D70F0EC112FEEC05F0C2EFF3
:1052CA0016F01200120012001200DBEF25F0120095
:1052DA0029EF26F06D840101080EF26F070EF36FB5
:1052EA00F207000EF35BF251F311FAE16D9412002A
:1052FA00D9CFE6FFE1CFD9FFFD0EDBCF22F0FE0EBC
:10530A00DBCF23F0720E221801E1235033E0E86864
:10531A00221802E17F0E23182BE0740E221801E1F5
:10532A00235024E0750E221801E123501DE0730E6C
:10533A00221801E1235016E0030E221801E123503E
:10534A000FE0020E221801E1235008E0010E221894
:10535A0001E1235001E010D0BBDF0FD0B8DF0DD040
:10536A00B4DF0BD0B0DF09D0ACDF07D0ABDF05D09C
:10537A00ABDF03D0000001D000D0010E00D0E5520F
:10538A00E7CFD9FF12001E0EF66E080EF76E000E5A
:10539A00F86E01010900F550ED6F0900F550EE6F46
:1053AA0003E1ED6701D03DD00900F550E86F09002F
:1053BA00F550E96F0900F550EA6F09000900F55048
:1053CA00E96E0900F550EA6E090009000900F55076
:1053DA00EB6F0900F550EC6F09000900F6CFEFF109
:1053EA00F7CFF0F1F8CFF1F1E8C1F6FFE9C1F7FF25
:1053FA00EAC1F8FF0101EB5302E1EC5307E00900AF
:10540A00F550EE6EEB07F8E2EC07F9D7EFC1F6FFBD
:10541A00F0C1F7FFF1C1F8FF0101ED07000EEE5BE5
:10542A00BFD71200FE0EE3CFE9FFFF0EE3CFEAFF7C
:10543A00E9CFF3FFEACFF4FFFB0EE35003E1FC0EE2
:10544A00E35009E0FB0EE30602E2FC0EE306FD0E62
:10545A00E350EE6EF1D71200FE0EE3CFE9FFFF0E26
:10546A00E3CFEAFFF36AF46AEE5203E0F34AF42A5E
:10547A00FBD71200FF0EE3CFF8FFE552FF0EE3CF92
:10548A00F7FFE552FF0EE3CFF6FFE552E66AE66A5A
:10549A00E66A0900F55209E0FD0EE32A05E1FE0E6F
:1054AA00E32A02E1FF0EE32AF4D7FD0EE3CF21F04F
:1054BA00FE0EE3CF22F0FF0EE3CF23F01200D9CF86
:1054CA00E6FFDACFE6FFE1CFD9FFE2CFDAFFE65215
:1054DA00E652E652E652D950FB0F2E6EFF0EDA2044
:1054EA002F6E2EC0DEFFDD6EDECFE6FFDDCFE6FFDC
:1054FA00FB0EDBCFE6FFFC0EDBCFE6FFFD0EDBCFBC
:10550A00E6FFF4C1E6FFF5C1E6FFE0EC1FF02E6E00
:10551A00070EE15C02E2E16AE552E16E2E50020EEC
:10552A00F3CFDBFF030EF4CFDBFF020EDBCF2EF04F
:10553A00030EDBCF2FF02EC0F3FF2FC0F4FF040EB3
:10554A00E15C02E2E16AE552E16EE552E5CFDAFF9B
:10555A00E7CFD9FF1200D9CFE6FFDACFE6FFE1CFD6
:10556A00D9FFE2CFDAFFFB0EDBCF2EF0FC0EDBCF4A
:10557A002FF00001800E2F141AE1FB0EDBCFE9FF9A
:10558A00FC0EDBCFEAFFEECFF3FFEDCFF4FFEE2AFE
:10559A00000EEF22F3CFE9FFF4CFEAFFFD0EDBCFD7
:1055AA00EFFFEF502F6AF36E2FC0F4FF10D0FB0EFF
:1055BA00DB50FE0806E1FD0EDBCFE6FFE4EC2BF044
:1055CA0005D0FD0EDBCFE6FFA1EC08F0E552E5526F
:1055DA00E5CFDAFFE7CFD9FF12001201000202007D
:1055EA000040D80492FD8201010200010902430031
:1055FA00020100C032090400000102020100052470
:10560A0000100104240202052406000105240100F9
:10561A00010705820308000209040100020A0000CA
:10562A00000705030240000007058302400000044A
:10563A0003090418035300630068006D0061006CDD
:10564A00007A0048006100750073000803550042A3
:0B565A00005700F65539563D565556D6
:1056660020502502F3CF1CF0F4CF1DF02602F35094
:105676001D26000EF4201E6E20502702F3501E2613
:10568600000EF4201F6E20502802F3501F262150D2
:105696002502F3501D26F4501E22000E1F22215013
:1056A6002602F3501E26F4501F2221502702F350E3
:1056B6001F2622502502F3501E26F4501F22225088
:1056C6002602F3501F2623502502F3501F261200F0
:1056D600FF0EE124E96EFF0EE220EA6EEDCFF4FF45
:1056E600EFCFF3FFF46607D0600EF36404D07B0EB1
:1056F600F36001D0F39A1200F36AF46AFF0EE12414
:10570600E96EFF0EE220EA6EED6607D02F0EEF641B
:1057160004D03A0EEF6001D0F32A12001F6A1E6A07
:105726001D6A1C6A200EE76ED89020362136223676
:1057360023361C361D361E361F3625501C5C265059
:105746001D5827501E5828501F5809E325501C5E27
:1057560026501D5A27501E5A28501F5A202AE72E17
:10576600E4D712004F4B0D0A000D0A005542572090
:10577600465720442056657273696F6E20312E3469
:055786002E370D0A00A2
:10578C00000EF36E00EE00F0080E01D81200EA6075
:10579C0002D0EE6AFCD7F350E9601200EE6AFCD737
:1057AC0016EE00F026EE00F0F86A1B9CC8EC29F00F
:1057BC0003EC04F057EC29F0FBD71200FF0EE3507A
:1057CC00ACBA04D0AF6AAB8EAC8A949CACA2FED7B8
:1057DC00AD6EF36EF46A1200FF0EE350E84E120049
:1057EC00000000D000D000D0E82EFAD712003031E3
:1057FC00323334353637383961626364656600009C
:10580C00000000000000000000000000000000008C
:10581C00000000000000000000000000000000007C
:10582C00000000000000000000000000000000006C
:10583C00000000000000000000000000000000005C
:0D584C00000000000000000000000000004F
:020000040030CA
:04000000E53EFFFEDC
:02000500F99B65
:06000800FFFFFF9FFFFF58
:00000001FF
